:0200000480007A
:100000006F008004732F2034930F80006308FF0378
:10001000930F90006304FF03930FB0006300FF038E
:10002000130F000063040F0067000F00732F2034CC
:1000300063540F006F00400093E19153171F0000BD
:1000400023223FFC6FF09FFF732540F163100500F2
:10005000970200009382020173905230735000188F
:10006000970200009382020273905230B702008020
:100070009382F2FF7390023B9302F0017390023A75
:1000800097020000938282017390523073502030A7
:1000900073503030735040309301000097020000DD
:1000A000938282F673905230130510001315F501F8
:1000B000634C05000F00F00F930110009308D0056A
:1000C000130500007300000093020000638E02001D
:1000D00073905210B7B20000938292107390223046
:1000E00073232030E39A62F47350003097020000CB
:1000F0009382420173901234732540F173002030D3
:100100009301200093020000170300001303030172
:10011000E70203006F00000C170300001303C3FF86
:10012000639A620A93014000130200001703000063
:1001300013030301E7060300631E300813021200D5
:1001400093022000E31452FE9301500013020000BA
:10015000170300001303430113000000E706030028
:10016000631A30061302120093022000E31252FEBB
:1001700093016000130200001703000013038301C2
:100180001300000013000000E706030063143004AE
:100190001302120093022000E31052FE930210009B
:1001A000170300001303C3016700C3FF938212000B
:1001B00093821200938212009382120093821200A3
:1001C00093821200930E4000930170006394D20159
:1001D000631030020F00F00F638001009391110053
:1001E00093E111009308D00513850100730000000E
:1001F0000F00F00F930110009308D00513050000C5
:1002000073000000731000C0000000000000000038
:1002100000000000000000000000000000000000DE
:1002200000000000000000000000000000000000CE
:0C023000000000000000000000000000C2
:1010000000000000000000000000000000000000E0
:1010100000000000000000000000000000000000D0
:1010200000000000000000000000000000000000C0
:1010300000000000000000000000000000000000B0
:081040000000000000000000A8
:040000058000000077
:00000001FF
